:020000040000FA
:100000001529820700341734243424342434173457
:100010000834373425342534253412340834343444
:100020001634213421342134083437342134213436
:100030002134163408343734253425342134083437
:10004000373424342434203408341634213425340D
:100050002534063408343734043404340434373453
:100060000834373408340234013401343634083467
:10007000373404340434123421340834373401342E
:100080000134013408341734203420341734203438
:1000900020341734083437341034043402343734FD
:1000A00008341634213425342334173408343734D3
:1000B00024342434103408341634213425342334C1
:1000C00017340834373424342434263411340834B3
:1000D00010342534253425340234083420342034B7
:1000E00037342034203408343634013401340134B8
:1000F00036340834343402340134023434340834AD
:1001000036340134013436340134013436340834A1
:10011000213411340434113421340834203410349F
:100120000734103420340834213423340434313477
:1001300021340834003400340834343408341034A2
:100140003734083403342534253425341134083445
:10015000253425342534123408340434143424343A
:100160003734043408343434253425342534023407
:100170000834163425342534253402340834213427
:1001800022342434303408341234253425342534D0
:100190001234083410342534253425341634083408
:1001A00082072934013478341934403498340134C6
:1001B000403423346034193401346C344034133403
:1001C00001348C344034003480346C3460348C34EA
:1001D000403466344F34413419346C3429342E346D
:1001E000493423344034493419347E3440340034A3
:1001F00080340130A100A00BFB28A10BFB280034A8
:10020000F030A000A00B022900344030A100A00B68
:100210000729A10B072900344030A200A00B0E29AA
:10022000A10B0E29A20B0E29003483168630810003
:100230000730990008308500831285011F2903309B
:10024000A9000430A700A8012808A40085192429C2
:10025000052105212408D020A300803A03194D2947
:100260002408D020403A03194029230801208500A2
:10027000083A03194829F92085010021A30A3529E4
:100280000521A70B2429240AA8000430A70024294B
:10029000F920F920F920A40A2A29A90B2329240AE4
:0802A000A8000330A900242985
:0207FE00900069
:02400E00843FED
:00000001FF
